:1000000041C0189518951895189518951895189534
:100010001895189569D001E007BB04E106BF00E020
:1000200002BF0BE80FBD03E003BF03E407B900E81C
:1000300006B908E004BB05E107BB00EC06B924B132
:1000400030E015B100E0020F131F212F220F220B09
:10005000322FC801D901082F092B0A2B0B2B11F4C1
:1000600081E090E0FC0175972CF08C0145E150E0B7
:1000700028D006BF00E10A95F1F700C0DECF0000EE
:100080008895FECF0FE90DBFC0E833D0C3DFF7DF9F
:10009000F6CF00241124EFE0001F111F001C111CDB
:1000A0000416150610F0041A150AEA95AAF7001F9F
:1000B000111FA0010095109508955195419550404C
:1000C0000895FF27552312F4F160F7DF112312F48E
:1000D000F09506D0DEDFF0FD03D0F1FDEECF089500
:1000E0001195019510400895BA93AA939A938A9313
:0600F000089501E00895EF
:00000001FF
:00000001FF
